:02000000D02806
:100008008C00030E8D0083120616963023200515EA
:100018000F0823200F0823200F082320051106129C
:10002800643081000B110D0E83008C0E0C0E09003C
:10003800FF008A017F080139820700340034FF3E3F
:10004800031D232800000800FF0083120613FF0188
:1000580008307F0203183D281E30FF00FF0B3228AE
:10006800000083127F1C06137F180617FF0CFF0A77
:100078002C281E30FF00FF0B3F28000083120617B4
:100088001E30FF00FF0B4628000008007F081C20D8
:10009800003A0319CF287F081C20253A031DCA28D7
:1000A800FF0A7F081C20633A03196128103A0319D4
:1000B8006628173A03197128CD287F08840000089C
:1000C8002820CD287F08840000080319CD287F0840
:1000D800840000082820FF0A66287F08840000089A
:1000E800FF00FF01FF1F7F28FF09FF09FF0A03190F
:1000F800FF0A2D3028200530FF0096017F08FF00F9
:100108007F08FF00FF01FF011030FF00FF0DFF0D0A
:10011800FF0D031893280A307F02031C95280A3024
:10012800FF02FF0B8A283030FF070318FF0A103040
:100138007F0784007F0880007F08FF007F08FF009A
:10014800FF011030FF00FF0DFF0DFF0D0318B02851
:100158000A307F02031CB3280A30FF020314FF0D84
:10016800FF0DFF0BA728FF037F087F04031D8228CC
:10017800FF0A10307F07840000080319CD281030CB
:100188007F07840000082820FF0ABD287F081C205C
:100198002820FF0A4A280800FB30831685008601BC
:1001A800063081008B168B178312051186140612F0
:1001B80078308F00643081008B13831286100430EE
:1001C800232086140330232001308E008312051C5F
:1001D800F1288E0A0E302320EA280E088F008B178C
:0201E800E0280D
:02400E00F13F80
:00000001FF
